:100000000C94E2000C940A010C940A010C940A016D
:100010000C940A010C940A010C940A010C940A0134
:100020000C940A010C940A010C9491060C9423057B
:100030000C940A010C940A010C940A010C940A0114
:100040000C940A010C940A010C940A010C940A0104
:100050000C940A010C940A010C940A010C942401DA
:100060000C940A010C940A010C940A010C940A01E4
:100070000C940A010C940A010C940A010C940A01D4
:100080000C940A010C940A010C940A010C940A01C4
:100090000C940A010C940A010C940A010C940A01B4
:1000A0000C940A010C940A010C940A0139023C02D6
:1000B0002B022F0235025D025D025D024002440206
:1000C00048024E0252025D0258020000000200097E
:1000D0000F0000030401000C0000000000000000FD
:1000E0000000000000000000000408020110408031
:1000F000401020408040800802040180402010020F
:10010000011080102040402004040404040304056E
:1001100002020202040302020202060606060606A4
:100120000404020202040400000000250028002B41
:10013000002E00310000000000240027002A002DBE
:1001400000300012010002EF0201404F1B08920034
:10015000010102030112010002000000404F1B08D0
:1001600092000101020301537061726B46756E00CB
:100170004C696C79506164205553420004030904B2
:10018000080B000202020100090400000102020043
:1001900000052400100105240101010424020605C4
:1001A0002406000107058103100040090401000234
:1001B0000A00000007050202400000070583024014
:1001C0000000220811241FBECFEFDAE0DEBFCDBF52
:1001D00011E0A0E0B1E0E4ECF1E102C005900D9285
:1001E000A432B107D9F721E0A4E2B1E001C01D9229
:1001F000A539B207E1F711E0C4ECD1E004C02297C1
:10020000FE010E94DC08C23CD107C9F70E94CE0261
:100210000C94E0080C94000061E08DE00C945E0208
:1002200061E08DE00E94970268EE73E080E090E06C
:100230000E94910160E08DE00E94970268EE73E0F9
:1002400080E090E00C9491011F920F920FB60F92F4
:1002500011242F933F938F939F93AF93BF938091DC
:10026000250190912601A0912701B091280130919C
:10027000240126E0230F2D3720F40296A11DB11D85
:1002800005C029E8230F0396A11DB11D2093240169
:100290008093250190932601A0932701B093280114
:1002A0008091290190912A01A0912B01B0912C01FC
:1002B0000196A11DB11D8093290190932A01A0935D
:1002C0002B01B0932C01BF91AF919F918F913F91E2
:1002D0002F910F900FBE0F901F9018953FB7F89475
:1002E0008091290190912A01A0912B01B0912C01BC
:1002F00026B5A89B05C02F3F19F00196A11DB11D81
:100300003FBF6627782F892F9A2F620F711D811D9D
:10031000911D43E0660F771F881F991F4A95D1F7FB
:1003200008958F929F92AF92BF92CF92DF92EF92F9
:10033000FF926B017C010E946E014B015C01C114B4
:10034000D104E104F104F1F00E94E1020E946E0187
:10035000681979098A099B09683E734081059105EE
:1003600070F321E0C21AD108E108F10888EE880E86
:1003700083E0981EA11CB11CC114D104E104F10456
:1003800029F7DDCFFF90EF90DF90CF90BF90AF9037
:100390009F908F900895789484B5826084BD84B5D1
:1003A000816084BD85B5826085BD85B5816085BD70
:1003B000EEE6F0E0808181608083E1E8F0E0108289
:1003C000808182608083808181608083E0E8F0E0CA
:1003D000808181608083E1E9F0E0808182608083B8
:1003E000808181608083E0E9F0E0808181608083AA
:1003F000E1ECF0E080818460808380818260808392
:10040000808181608083E3ECF0E080818160808383
:10041000E0ECF0E0808182608083E2ECF0E08081BB
:1004200081608083EAE7F0E080818460808380815E
:100430008260808380818E7F8083808180688083DA
:10044000089590E0FC013197EF30F105B0F5EA5ADC
:10045000FF4F0C94DA08809180008F7703C0809161
:1004600080008F7D80938000089580918000877F39
:10047000F9CF84B58F7702C084B58F7D84BD089590
:10048000809190008F7707C0809190008F7D03C08E
:1004900080919000877F8093900008958091C000A4
:1004A0008F7703C08091C0008F7D8093C000089536
:1004B0008091C200877F8093C2000895CF93DF931D
:1004C00090E0FC01E751FF4F2491FC01E85FFE4FF3
:1004D0008491882349F190E0880F991FFC01EB5C1F
:1004E000FE4FA591B491895D9E4FFC01C591D491B9
:1004F0009FB7611108C0F8948C91209582238C934A
:10050000888182230AC0623051F4F8948C91322F92
:10051000309583238C938881822B888304C0F89440
:100520008C91822B8C939FBFDF91CF9108950F9375
:100530001F93CF93DF931F92CDB7DEB7282F30E004
:10054000F901E653FF4F8491F901E751FF4F1491F0
:10055000F901E85FFE4F04910023C9F0882321F0E0
:1005600069830E9421026981E02FF0E0EE0FFF1FF6
:10057000E95DFE4FA591B4919FB7F8948C916111FC
:1005800003C01095812301C0812B8C939FBF0F90D6
:10059000DF91CF911F910F91089508950E94CB0193
:1005A0000E94CD028DE291E00E9414070E940C018E
:1005B000C0E0D0E00E9410012097E1F30E9400000B
:1005C000F9CF0895615030F02091F100FC012083B3
:1005D0000196F8CF289884E68093360108954091DB
:1005E00031015091320120912F0130913001421799
:1005F0005307B4F49091E8009570E1F39091E8000E
:1006000092FD19C08093F1008091310190913201E7
:1006100001968F739927892B19F48EEF8093E80048
:100620008091310190913201019690933201809333
:10063000310181E0089580E00895CF92DF92EF923A
:10064000FF920F931F93CF93DF931F92CDB7DEB727
:10065000082F162FF42E862F880F8E5F99830E9405
:10066000EF0283E00E94EF02E02EC02E9981D92E86
:100670008C2D8E19811798F4F601F7FE02C0849133
:1006800001C080810E94EF02082F80E00E94EF02EB
:100690008023FFEFCF1ADF0A8111EACF01C081E08A
:1006A0000F90DF91CF911F910F91FF90EF90DF900E
:1006B000CF9008958091D70081608093D70080EA21
:1006C0008093D80089B58F7E89BD89B5826089BD48
:1006D00009B400FEFDCF61E070E080E090E00E9490
:1006E00091018091D8008F7C80618093D8008091A7
:1006F000E000807F8093E0000895CF93DF931F9206
:10070000CDB7DEB71982CE0101960E948E070E94F6
:10071000C608BE016F5F7F4F0E943F0889810F901E
:10072000DF91CF9108952FB7FC012083F894677073
:100730006093E9000895CF93DF931F92CDB7DEB7A2
:10074000682FCE0101960E9493038091F200998157
:100750009FBF0F90DF91CF910895FF920F931F934A
:10076000CF93DF9300D0CDB7DEB7F62E8A019091FC
:100770003501992311F057FF03C08FEF9FEF2BC076
:10078000682FCE0101967A830E9493038091F20034
:1007900090E0A8017A81801791070CF4AC01EF2D4D
:1007A000F72FF40E84E6FE1639F028988093360170
:1007B0009091F1009193F7CF4115510521F080916F
:1007C000F200882321F089818FBFCA0104C08BE623
:1007D0008093E800F8CF0F900F90DF91CF911F9199
:1007E0000F91FF900895CF93DF931F92CDB7DEB79F
:1007F00041E050E0BE016F5F7F4F0E94AD03019763
:1008000019F4898190E002C08FEF9FEF0F90DF9184
:10081000CF910895CF93DF931F92CDB7DEB7682FA6
:10082000CE0101960E9493039091E800892F807277
:1008300095FF04C09091F20080E4891B99819FBFCD
:100840000F90DF91CF9108956F927F928F929F9238
:10085000AF92BF92CF92DF92EF92FF920F931F93CE
:10086000CF93DF931F92CDB7DEB7782E7B01C42ED6
:10087000B52E80913501882369F0042F152F8AEF5A
:10088000D82E872D8072982E9AE3A92E872D8074FA
:10089000882E11C08FEF9FEF57C0872D0E940A044A
:1008A000682E81110CC0DA94A9F361E070E080E059
:1008B00090E00E9491010115110579F73BC0282FA6
:1008C00030E0021713070CF4602E672DCE0101965D
:1008D0000E9493038091E80085FF29C0262D30E017
:1008E000021B130B992039F06A948FEF6816B1F050
:1008F0001092F100F9CFF701862D77FE07C08150E5
:1009000058F094919093F1003196F9CF815020F0F6
:1009100091919093F100FACFE20EF31E8091E800DE
:1009200085FF0FC00115110511F481100AC08981DE
:100930008FBFC1CF5D9884E6809337018C2D9B2DAE
:1009400003C0A092E800F3CF0F90DF91CF911F91E9
:100950000F91FF90EF90DF90CF90BF90AF909F905E
:100960008F907F906F9008951092E900109232015D
:10097000109231019093300180932F010895CF920E
:10098000DF92FF920F931F93CF93DF9300D0CDB7E9
:10099000DEB7F82E8A016B0101151105B1F0F601E1
:1009A000F7FE02C0849101C0808149835A830E946E
:1009B000EF0201501109FFEFCF1ADF0A49815A8176
:1009C0008111EACF8FEF9FEF01C0CA010F900F9006
:1009D000DF91CF911F910F91FF90DF90CF900895FD
:1009E000BF92CF92DF92EF92FF920F931F93CF931C
:1009F000DF936C018B01EB013BEFB32E2097C1F02D
:100A00007E01C134D1051CF020E4E22EF12C80914E
:100A1000E80082FFFCCFC8018C1B9D0B6E2D8C0D56
:100A20009D1D0E94E202B092E800CE19DF09E6CFD8
:100A3000C801DF91CF911F910F91FF90EF90DF9050
:100A4000CF90BF9008951F920F920FB60F9211246E
:100A5000DF92EF92FF920F931F932F933F934F9349
:100A60005F936F937F938F939F93AF93BF93EF9316
:100A7000FF93CF93DF93CDB7DEB76C97DEBFCDBFCB
:100A80001092E9008091E80083FF23C168E0CE0165
:100A900045960E94E20282EF8093E8003D8937FF8D
:100AA00005C08091E80080FFFCCF03C08EEF8093EB
:100AB000E800832F807609F0F0C02E894F89D88C0A
:100AC00021110CC0303829F4809134018093F10059
:100AD00002C01092F1001092F100F4C0842F90E057
:100AE0009D29213049F43111EDC0019709F0EAC088
:100AF000809134018D7F0AC0233059F43111E2C056
:100B0000019709F0DFC08091340182608093340145
:100B1000D9C0253041F48091E80080FFFCCF4068C7
:100B20004093E300CFC0263009F08DC0EB8CFC8CE5
:100B300022E0D2122CC080E090E00E94B4040E9417
:100B40007D0399E08E010F5F1F4FF801292F11924D
:100B50002A95E9F79983DA8291E09E8390EA988753
:100B60009AEF99872091310130913201275F3F4FF1
:100B70003C832B838D83C7010E94B40449E050E07D
:100B8000B80180E00E94BF040E947D039BC0C701A2
:100B90000E94B4040E94C608BE016B5E7F4F0E9493
:100BA0006808009719F00CF08DC090C081E0D81251
:100BB0000EC08B8D9C8D089719F481E080932E01D7
:100BC00080912E0181112FC065E571E031C0E3E015
:100BD000DE127CC08F89882349F1823029F440E8F5
:100BE0006BE080E791E01CC0813029F440E868E0C8
:100BF00087E691E015C0833009F068C00E94C608FE
:100C00008E010F5F1F4FB8010E948708F801019005
:100C10000020E9F73197E01BF10B40E06E2FC8018F
:100C20000E941D034DC063E471E002C06CE771E0F7
:100C30006115710509F44AC0FB01449150E080E858
:100C40000E94BF043FC0273009F440C0283021F47F
:100C500081E08093F10036C02930A1F53370B1F501
:100C6000E1E0F1E081E021E036E39081992361F059
:100C70008093E9002093EB0091919093EC003093E6
:100C8000ED008F5F873089F78EE78093EA0010923E
:100C9000EA008F898093350115C08B8D9C8D0E9451
:100CA000B404898D811105C0CE0145960E94990733
:100CB00007C00E94C608BE016B5E7F4F0E94A60857
:100CC000882321F08EEF8093E80003C081E28093B7
:100CD000EB006C960FB6F894DEBF0FBECDBFDF9170
:100CE000CF91FF91EF91BF91AF919F918F917F91A4
:100CF0006F915F914F913F912F911F910F91FF90B5
:100D0000EF90DF900F900FBE0F901F90189580937B
:100D1000E9008091F200882319F08AE38093E800CB
:100D200008951F920F920FB60F9211242F933F93A5
:100D30004F935F936F937F938F939F93AF93BF93E3
:100D4000CF93EF93FF93C091E1008091E100837F07
:100D50008093E1008093E100C3FF0FC01092E9008F
:100D600081E08093EB001092EC0082E38093ED0031
:100D70001092350188E08093F000C2FF19C083E033
:100D80000E94870680913701882339F080913701CE
:100D9000815080933701882389F18091360188231F
:100DA00039F080913601815080933601882341F1DA
:100DB000C4FF10C08091E2008E7E81608093E200CB
:100DC0008091E1008F7E8093E100809133018E7EDF
:100DD000806111C0C0FF16C08091E2008E7E8061EC
:100DE0008093E2008091E1008E7E8093E10080910B
:100DF00033018E7E81608093330104C05D9ACDCF34
:100E0000289AD6CFFF91EF91CF91BF91AF919F914B
:100E10008F917F916F915F914F913F912F910F90A3
:100E20000FBE0F901F90189510923501109234014B
:100E3000109233010E945A038091E1008E7E8093CC
:100E4000E1008DE08093E200559A209AEEEFFFE7F3
:100E5000859194918B3F9C4D19F481E0809388019A
:100E60000895CF93DF931F92CDB7DEB76983DC017E
:100E7000ED91FC910280F381E02D41E050E0BE0154
:100E80006F5F7F4F09950F90DF91CF910895CF93BA
:100E9000DF93EC018C859D8597FF05C082E00E9461
:100EA000F3039D878C878C859D85DF91CF91089575
:100EB00083E00C948706FC018485958597FD06C028
:100EC00082E00E949B0390E00196089582E00E94D8
:100ED0009B0390E00895FC018485958597FD05C0EE
:100EE0002FEF3FEF35872487089582E00C94F303BA
:100EF000CF93DF93EC0180911201882331F083E0DE
:100F00000E9424041816190634F081E090E09B83B7
:100F10008A8380E090E0DF91CF910895FC012081E9
:100F20002E5F208342E450E060E871E080E80C949A
:100F3000BF04FC0121818081813A59F4213209F0FA
:100F40004BC047E050E06BE071E080E00E94BF04DE
:100F50005EC0813209F040C0233289F4838190E081
:100F6000982F88273281832BA0E0B0E0809307017F
:100F700090930801A0930901B0930A010FC0203299
:100F800039F467E070E08BE091E00E94F00409C062
:100F9000223221F482818093120103C02D7F2032FE
:100FA000B1F580918801811103C0E0E0F8E002C052
:100FB000EEEFFAE080910B0190910C01A0910D01F0
:100FC000B0910E01803B9440A105B10511F58091CF
:100FD000120180FF03C01DC080E00895EE3F2AE0AB
:100FE000F20731F0808191819093FF0A8093FE0A8D
:100FF00087E797E7918380832BE088E190E00FB645
:10100000F894A895809360000FBE2093600081E063
:10101000089588E10FB6F894809360001092600004
:101020000FBEA895EE3F8AE0F80739F08091FE0ADE
:101030009091FF0A91838083EACF1092FF0A109269
:10104000FE0AE5CF10923B0110923A0188EE93E040
:10105000A0E0B0E080933C0190933D01A0933E015D
:10106000B0933F0187E191E090933901809338017B
:101070008FEF9FEF90934501809344010895EF9285
:10108000FF920F931F93CF93DF937B01FC01C281EB
:10109000D38100E010E0209781F0E881F98102809F
:1010A000F381E02DB701CE01099597FD08C0080F27
:1010B000191F0884D985C02DEECFC80102C08FEF5B
:1010C0009FEFDF91CF911F910F91FF90EF900895C7
:1010D0000F931F93CF93DF938B01FC01C281D381C8
:1010E000209771F0E881F9810480F581E02DB80145
:1010F000CE010995009731F40884D985C02DF0CF31
:1011000080E090E0DF91CF911F910F9108950F93B0
:101110001F93CF93DF938B01FC01C281D381209772
:1011200071F0E881F9810680F781E02DB801CE01E8
:101130000995080F111D0884D985C02DF0CFF8013D
:101140001082DF91CF911F910F9108950F931F93FC
:10115000CF93DF938B01FC01C281D381209771F083
:10116000E881F9810190F081E02DB801CE01099567
:10117000811106C00884D985C02DF0CF80E001C060
:1011800081E0DF91CF911F910F91089580918D01A2
:1011900081110DC082E08093890184E080938A01EF
:1011A00010928C0110928B0181E080938D0189E86F
:1011B00091E00895EE0FFF1F0590F491E02D099442
:0411C000F894FFCFD1
:1011C40000C18081000000FFFFFFFF00E10000007C
:1011D40000000000000000310778075B076B074739
:0411E40007580700A1
:00000001FF
